:020000040800F2
:1000000000250020550200089D200008591F000807
:10001000992000083D050008192A0008000000008A
:100020000000000000000000000000000D28000893
:10003000FD05000800000000D92000081128000874
:100040006F0200086F0200086F0200086F020008CC
:100050006F0200086F0200086F0200086F020008BC
:100060006F0200086F0200086F0200086F020008AC
:100070006F0200086F0200086F0200086F0200089C
:100080006F0200086F0200086F0200086F0200088C
:10009000410500086F0200086F0200086F020008A7
:1000A0006F0200086F0200086F0200086F0200086C
:1000B000D12800086F0200086F0200086F020008D4
:1000C0006F0200086F0200086F0200086F0200084C
:1000D0006F0200086F0200086F0200086F0200083C
:1000E0006F0200086F0200086F0200086F0200082C
:1000F0006F0200086F0200086F0200086F0200081C
:100100006F0200086F0200086F0200086F0200080B
:100110006F0200086F0200086F0200086F020008FB
:100120006F0200086F0200086F0200086F020008EB
:100130006F02000800000000000000006F020008CD
:100140006F0200086F0200086F0200086F020008CB
:100150006F0200086F0200086F0200086F020008BB
:100160006F0200086F0200086F0200086F020008AB
:100170006F0200086F02000800000000000000008D
:100180006F0200086F02000800F002F800F052F859
:1001900014A696E8000CB244B344DA4501D100F04D
:1001A00049F8BAE80F000FA696E83000A5EB040561
:1001B00004EB0607AAEB0704A7F101074FEA1515A0
:1001C0004FEA3414A4F10104AC4201D300F032F838
:1001D00013F0010F18BFFB1A43F0010300F001F800
:1001E000DBE71847EC4200000C430000103A24BF44
:1001F00078C878C1FAD8520724BF30C830C144BF8C
:1002000004680C6070470000704700000023002461
:1002100000250026103A28BF78C1FBD8520728BF16
:1002200030C148BF0B6070471FB503F02AFF1FBDE8
:1002300010B510BD00F047F91146FFF7F5FF03F0C8
:10024000C7FE00F065F903B4FFF7F2FF03BC00F04E
:100250006DF900000948804709480047FEE7FEE7BE
:10026000FEE7FEE7FEE7FEE7FEE7FEE7FEE7FEE766
:1002700004480549054A064B70470000BD280008A0
:1002800089010008001F0020002500200021002017
:100290000021002053EA020C00F069802DE9F04BA8
:1002A0004FF00006002B1FBFB3FA83F503FA05F4E5
:1002B00024FA05F65E4012BF1643B2FA82F502FA3E
:1002C00005F4C5F120051EBF22FA05FC44EA0C0422
:1002D000203556EA044C4FEA144418BF641C4FF012
:1002E00000084FF00009904271EB030C39D300294C
:1002F00019BFB1FA81F701FA07F6B0FA80F700FAF0
:1003000007F6C7F120071EBF20FA07FC46EA0C06D5
:100310002037B6FBF4FCA7EB0507103F07F01F0BD7
:10032000CBF120062CFA06F60CFA0BFB44BFB346C1
:100330000026202FA4BF5E464FF0000B5BEA060CA0
:1003400008BF4FF0010B19EB0B0948EB0608ABFB9C
:10035000027C06FB02CC0BFB03CCC01B71EB0C0137
:10036000C1E70B46024641464846BDE8F08B13B54F
:10037000084318BF4FF0FF300146AFF30080BDE8DF
:100380001C407047032A40F2308010F0030C00F04C
:10039000158011F8013BBCF1020F624498BF11F8BF
:1003A00001CB00F8013B38BF11F8013BA2F1040278
:1003B00098BF00F801CB38BF00F8013B11F00303F0
:1003C00000F04F80083AC0F0088051F8043B083A2A
:1003D00051F804CBA0E80810F5E7121D5CBF51F8F6
:1003E000043B40F8043BAFF30080D20724BF11F870
:1003F000013B11F801CB48BF11F8012B24BF00F8D5
:10040000013B00F801CB48BF00F8012B70474FF0CB
:10041000000200B5134694469646203922BFA0E854
:100420000C50A0E80C50B1F12001BFF4F7AF090760
:1004300028BFA0E80C5048BF0CC05DF804EB890051
:1004400028BF40F8042B08BF704748BF20F8022B94
:1004500011F0804F18BF00F8012B704770477047AC
:10046000704710B5203AC0F00B80B1E81850A0E8F2
:100470001850B1E81850A0E81850203ABFF4F5AF72
:100480005FEA027C24BFB1E81850A0E8185044BFCE
:1004900018C918C0BDE810405FEA827C24BF51F83B
:1004A000043B40F8043B08BF7047D20728BF31F82F
:1004B000023B48BF11F8012B28BF20F8023B48BF80
:1004C00000F8012B7047754600F02CF8AE46050089
:1004D0006946534620F00700854618B020B5FFF75F
:1004E000C7FEBDE820404FF000064FF000074FF078
:1004F00000084FF0000BAC46ACE8C009ACE8C009FE
:10050000ACE8C009ACE8C00921F007018D4670478E
:1005100010B50446AFF300802046BDE81040FFF759
:1005200092BE0000004870471800002001491820C2
:10053000ABBEFEE72600020070470000FEE70000A9
:1005400040F2F800C2F2000000F03ABA10B58AB0EA
:100550000020CDE90500CDE90000CDE902000490BE
:100560000E20099040F2C400C2F20000012100F107
:100570003404CDE907116946204600F0DBF8002875
:1005800018BF00F03DF8204600F064FC2046022130
:1005900000F066F80AB010BDF0B581B0069F1E46A7
:1005A000154600F075FE40F2C40104460120C2F277
:1005B0000001009004200022082F28BF0827C1E96D
:1005C000005501F1080301F1340585C36B46284647
:1005D000324600F05DF800BF0099284600F09AFB13
:1005E00050B100F055FE001B6528F5D30099284650
:1005F00000F00AF8F0E700BF01B0F0BD704700005E
:1006000072B600BFFEE7000090F82020013A012AF0
:100610001CD8CA0704D00268936843F08003936033
:100620008A0704D50268936843F40043936049073E
:100630005CBF0020704700684FF4000200F1080121
:1006400000200B681A430A60704700BF00F12401C4
:1006500001204FF480220B681A430A6070470000A3
:1006600090F82020013A012A08D8006800F114020D
:100670000020136819431160704700BF00F1240285
:1006800001204FF480211368194311607047000066
:1006900010B590F820E0D0F800C0AEF1010EBEF128
:1006A000010FDCF808E011D81EF0E05F18D0CEF39F
:1006B00001640120A04018608B68DBB1D1F804E030
:1006C000C86840EACE0040EA030E17E000F12403B8
:1006D00001204FF480211A681143196010BD00BF3A
:1006E00000F1240301204FF400111A68114319602E
:1006F00010BD00BF0868CB6843EA405E0CF5C070CF
:1007000000EB0413240140F804E00C69184640F89B
:10071000044F097D012903D1016841F48071016012
:1007200050680121D8601068986000201A68114351
:10073000196010BD90F82020013A012A30D8B0B5D8
:1007400046F20060C4F20000026842F0010202605A
:10075000026822F47C520260D1F814E0CC694A6A43
:100760000368012C43EA022202600EF01F024FF0E0
:10077000010303FA02F2C3696FEA020C23EA0203DF
:10078000C36113D02CBBC36803EA0C03C360CB68FE
:100790008C8844EA034300EBCE0423640B4611E04B
:1007A000416A41F48021416201207047C3681343CC
:1007B000C3600B688C8844EA034300EBCE042364D7
:1007C00001F10C038C681B8843EA044300EBCE0460
:1007D000636443688D6943EA0204D1F810E0096A52
:1007E000002D08BF03EA0C0444604369BEF1000F0A
:1007F00043EA020408BF03EA0C040129446102D160
:10080000C1691143C161016821F00101016000204B
:10081000B0BD0000002804BF01207047B0B50446F9
:1008200090F82000022817D12068016841F00101EA
:10083000016000F02DFD054620684168C90711D10F
:1008400000F026FD401B0B28F6D3606A40F4003010
:10085000606205200BE000BF606A40F480106062B7
:1008600007E000BF016821F002010160012084F867
:100870002000204600F05EFA2068016841F4004143
:1008800001600020606284F82000B0BD7047000065
:10089000B0B590F82040013C012C7DD8D0F800C0C4
:1008A00000290CBFDCF80C40DCF81040A4077DD018
:1008B0000CF5D8754FEA011C55F80C4014F00404EF
:1008C000946055F80CE005EB011C19BF4FEADE05FA
:1008D00055604FEA5E551560DCF80050E64605F0BD
:1008E0000205D5605EF8044F24075ABFDEF80040C9
:1008F00004F00F0408241461DEF800400029C4F35A
:1009000007249461DEF800504FEA15455561DCF884
:1009100008201A70026802EB0112D2F8B8214FEADF
:1009200012225A70026802EB0112D2F8B8214FEA83
:1009300012429A70026802EB0112D2F8B8214FEA13
:100940001262DA70026802EB0112D2F8BC211A714D
:10095000026802EB0112D2F8BC214FEA12225A714E
:10096000026802EB0112D2F8BC214FEA12429A71DE
:10097000026802EB0112D2F8BC214FEA1262DA716E
:1009800000680CBF00F10C0100F1100100202022D2
:100990000B681A430A60B0BD00F1240101204FF436
:1009A00080220B681A430A60B0BD00BF00F1240129
:1009B00001204FF400120B681A430A60B0BD00001A
:1009C0002DE9F04F81B0044600684669D0F80490E4
:1009D0008768D0F80CB0D0F810A0D0F81880F107D4
:1009E00004D1002530071DD424E000BFF90710D042
:1009F0000121BA07816009D4780700F1AF80380778
:100A000000F1B680204600F053FA02E0204600F0E4
:100A100051FA0025F80500F18780F80300F1B18054
:100A2000300707D51BF0100004D0206845F400758E
:100A30001021C160700708D51BF0080005D02068A0
:100A40000821C160204600F0D5F9B00706D520681E
:100A5000C068800702D0204600F0CEF9700607D5A6
:100A60001AF0100004D0206845F48065102101615F
:100A7000B00608D51AF0080005D0206808210161E9
:100A8000204600F0E1F9F00606D5206800698007ED
:100A900002D0204600F0DAF9B00308D519F01000B2
:100AA00005D0206810214160204600F0D1F9F00304
:100AB00008D519F0080005D02068082141602046BB
:100AC00000F002FA300440F19B805FEA497040F187
:100AD000948006F4807008EA102028435FEA887149
:100AE000014648BF41F00201B20558BF01465FEA26
:100AF00048700D4648BF45F00405700558BF0D46C7
:100B0000300540F17A8018F0700000F076801038DF
:100B1000000905286CD8DFE800F003655D615969BC
:100B200045F0080564E000BF20684FF48071BA0505
:100B300081600BD4780515D438051DD4204600F00B
:100B4000BBF9F8037FF56CAF1BE000BF204600F057
:100B5000B5F9F8037FF564AF13E000BF4FF400650B
:100B600058E700BF05F50055F8037FF559AF08E0D9
:100B70004FF480554EE700BF05F58045F8037FF53B
:100B80004FAF20684FF48031BA0381600AD47803F4
:100B900010D4380314D4204600F092F930073FF502
:100BA00041AF47E7204600F08DF930073FF53AAFF7
:100BB00040E700BF05F5004530073FF533AF39E7A3
:100BC00005F5803530073FF52DAF33E745F080055B
:100BD0000EE000BF45F020050AE000BF45F04005EB
:100BE00006E000BF45F0100502E000BF45F4807547
:100BF0002068816921F070018161206804214160D1
:100C000055B1606A40EA05012046616201B0BDE865
:100C1000F04FFFF73BBE00BF01B0BDE8F08F000012
:100C2000002804BF01207047B0B5044690F82000AA
:100C300010B9204600F09AF82068016841F00101DF
:100C4000016000F025FB054620684168C90705D111
:100C500000F01EFB401B0B28F6D310E0016821F0CA
:100C60000201016000F014FB054600BF20684168E6
:100C700089070DD500F00CFB401B0B28F6D3606AEA
:100C8000052140F400306062012084F82010B0BDDE
:100C9000217E0268012922F0800208BF80320260B2
:100CA000617E0268012922F0400208BF40320260E2
:100CB000A17E0268012922F0200208BF20320260D2
:100CC000E17E0268012922F0100218BF1032026092
:100CD000217F0268012922F0080208BF0832026061
:100CE000617F0268012922F0040208BF0432026019
:100CF000D4E901C2D4E9033561691A432A43114397
:100D0000ACF101021143C16100200121606284F84D
:100D10002010B0BD90F82020013A012A84BF0020A5
:100D200070470068806800EA8160B0EB816018BF9E
:100D300001207047016846F20040C4F20000814281
:100D400018BF704780B543F64001C4F202010A683B
:100D500000F5D03022F000720A604FF4407100F0CC
:100D6000D7F81420BDE8804000F004BB80B586B001
:100D700046F200410068C4F2000100228842059258
:100D8000CDE903220292019202D006B080BD00BFDD
:100D900043F630000092C4F20200036943F000738E
:100DA0000361036903F000730093009B00920368E2
:100DB00043F002030360006800F002000090009816
:100DC0004FF4407001900220CDE90202032004900C
:100DD0000920059001F5D03001A900F083F9142015
:100DE0000021002200F0EEFA142000F0D9FA06B03B
:100DF00080BD000070470000006846F20041C4F268
:100E00000001884218BF704710B582B040F2C40498
:100E1000C2F2000404F1340004F118026B46002110
:100E2000FFF736FDE06940F20171884208D1206A7F
:100E3000042805D194F828306A46002001F0BCFE51
:100E400002B0BDE8104070477047000070470000D6
:100E500070470000B0B5044690F8200001281DD16D
:100E6000022084F820002068016821F0010101605F
:100E700000F00EFA054600BF20684068C00713D096
:100E800000F006FA401B0B28F6D3606A40F40030ED
:100E90006062052084F820000120B0BD606A40F443
:100EA000002060620120B0BD00206062B0BD000083
:100EB0007047000070470000704700007047000056
:100EC00070470000704700007047000080B543F68F
:100ED00010004CF6FF11C4F20200CFF2FE6147F69B
:100EE000331201610021C0F277420161426141F297
:100EF000FF12C2F2600241610260C12201604260E1
:100F0000012241608260816000F016FA002080BDFD
:100F10002DE9F04F82B000F13E4241F6004789468C
:100F200002F1FF72C4F2020708214FEAB223B8426D
:100F300008BF072100F12007002404254FF0020B11
:100F40000097072B38BF4FEAB221019126E000BF7E
:100F50000168032202FA0BF2914301606FF0030172
:100F6000009F01EA540305F01C0CFE580F2101FA02
:100F70000CF126EA0101F950C168D1469143C160E4
:100F8000416821EA0E014160816891438160023429
:100F90000835102C0BF1040B00F0A080012101FAA0
:100FA00004F818EA090A59D043F60041C4F20101D5
:100FB0002F1FA1F57E7C24F0030207F0080E0F21FD
:100FC0005CF8023001FA0EF20199134001FA0EF6B4
:100FD000B34224D143F6004EC4F2010EDEF80030D5
:100FE00043F60C4123EA0A03CEF80030DEF8043061
:100FF000C4F2010123EA0A03CEF804300B68A60804
:1010000023EA0A030B60DEF8083023EA0A03CEF86D
:1010100008305CF8263023EA02024CF82620ABF1B7
:1010200002020368032101FA02F29343036007F00E
:10103000180C6FF00301009F01EA5406B9590F2301
:1010400003FA0CF39943B951C1689143C1604168F7
:1010500021EA08014160816891438160022101FA1F
:1010600004FE1EEA090292D043F60041C4F20101D7
:10107000CA46A1F57E7924F0030105F00C060F2382
:1010800059F8011003FA06FC019B01EA0C0103FA6E
:1010900006F6B1427FF45CAF43F60048C4F20108A3
:1010A000D8F8001043F60C469143C8F80010D8F861
:1010B0000410C4F201069143C8F80410316891434A
:1010C0003160D8F80810A6089143C8F8081059F8FC
:1010D000261021EA0C0149F8261039E702B0BDE8D4
:1010E000F08F00002DE9F04F83B000F1200200F1F5
:1010F0003E4741F60045009207F1FF77C4F2020532
:1011000008224FEAB726A84208BF072200254FF061
:1011100000084FF00009072E38BF4FEAB7220192AE
:101120000AE000BF09F1010908F10208B9F1100F46
:1011300005F1040500F0A2800F68012202FA09FE01
:1011400017EA0E0AEED0D1F804C003220CF0030710
:101150007E1E02FA08F4012E6FEA040B12D884688E
:10116000CE6804EA0B0406FA08F634438460446847
:1011700024EA0E06CCF3001404FA09F42643466070
:1011800004E000BF032F01D103271EE0C6688C686E
:1011900006EA0B0604FA08F42643022FC66014D1AF
:1011A0006FF00302009E02EA590756F807C005F0E7
:1011B0001C040F220B69A2402CEA0202A3401A432E
:1011C000F251D1F804C00CF00307026807FA08F3E3
:1011D00002EA0B021A431CF4403F0260A2D0002234
:1011E00043F644030292C4F202031A6843F6004431
:1011F00042F480421A601A68C4F2010402F4804288
:101200000292029A29F003024FF6084C2244CFF6CC
:10121000FF7C52F80C3005F00C070F26BE40B3439C
:10122000019E06FA07F73B4342F80C30A2684B6870
:1012300042EA0A0743F60C4CDE0258BF22EA0A07CC
:10124000A760C4F2010CDCF800209E0242EA0A0703
:1012500058BF22EA0A07CCF8007062689E0342EA8F
:101260000A0758BF22EA0A0767602268DB0342EADE
:101270000A0758BF22EA0A07276053E703B0BDE810
:10128000F08F0000002A08BF090481617047000048
:1012900041F6FC60C2F200000068704740F20000B6
:1012A00041F6FC61C2F20000C2F2000100780A6857
:1012B000104408607047000080B543F60040C4F257
:1012C0000200016841F400710160016841F480612D
:1012D0000160016841F480710160032000F09EF814
:1012E0000F2000F005F800F029F8002080BD000074
:1012F00070B540F20006C2F2000640F20C013278EE
:10130000C2F200014FF47A730968B3FBF2F20446AB
:10131000B1FBF2F1084600F051FB0F2C4FF0010534
:1013200008D838B94FF0FF3021460022002500F0E0
:1013300049F87460284670BD7047000082B00020F4
:1013400043F640010190C4F202014A6842F480422F
:101350004A604A6802F480420192019A009008684B
:1013600040F080500860086800F0805000900098BD
:1013700002B07047002848BF704700F01F010122EB
:1013800002FA01F11C2202EAD0004EF28012CEF2E3
:1013900000028150BFF34F8FBFF36F8F7047000083
:1013A000002848BF704700F01F01012202FA01F136
:1013B0001C2202EAD0004EF20012CEF2000281504E
:1013C0007047000010B54EF60C5CCEF2000CDCF855
:1013D0000030C3F3022E8EF00704042C28BF04242F
:1013E000BEF103034FF0FF3E0EFA04F438BF0023B2
:1013F000A14399400EFA03F39A43114300F00F0200
:1014000000F160430901043A03F564436244002893
:1014100048BF02F10C03197010BD00004EF60C51CC
:10142000CEF200010A684FF6FF031A4060F30A2269
:1014300042F0806040F0FD7008607047002804BFF3
:10144000012070472DE9F04143F60808C4F2020874
:101450000446D8F8F8030D4600F00700814207D98A
:1014600088F8F853D8F8F80300F00700A84277D1BD
:101470002068810717D5410705D5D8F8001041F439
:10148000E051C8F80010010705D5D8F8001041F464
:101490006041C8F80010D8F80010A26821F0F001EF
:1014A0001143C8F80010C00740D1D8F8F80300F085
:1014B0000700854207D288F8F853D8F8F80300F0FF
:1014C0000700A8424CD12068410707D5D8F8001082
:1014D000E26821F4E0511143C8F80010000708D574
:1014E000D8F80000216920F4604040EAC100C8F843
:1014F000000000F055F8D8F8001044F29C02C1F347
:101500000311C0F60002515C40F20C0220FA01F116
:1015100040F20400C2F200000068C2F20002116052
:10152000FFF7E6FE0020BDE8F08100BF6068811E85
:10153000022907D258F8081C89015CBF0120BDE8C8
:10154000F08111E0012807D158F8081C89035CBF1D
:101550000120BDE8F08107E058F8081C890703D492
:101560000120BDE8F08100BFD8F8001021F0030190
:101570000843C8F80000FFF78BFE064641F28837A3
:10158000D8F80000616800F00C00B0EB810F8CD03F
:10159000FFF77EFE801BB842F2D90320BDE8F08140
:1015A00010B543F60404C4F202046168C1F381017A
:1015B00042F20040C0F2F400DFE801F002040A0247
:1015C00010BD00BF41F20020C0F27A0010BD00BF84
:1015D000216801F03F02216823684902C3F38811A2
:1015E00006D4A1FB00010023FEF754FE07E000BF74
:1015F00041F20020C0F27A004843B0FBF2F02168CB
:101600000222C1F3014102EB4101B0FBF1F010BD38
:10161000002804BF012070472DE9F04182B0044644
:10162000007843F60006C007C4F202060CD0B0688A
:1016300000F00C00042840F081803068800303D55E
:101640006068002800F06881207880071BD5B068AA
:1016500010F00C0F09D0B06800F00C00082840F022
:1016600087807068400200F183803068800703D56E
:10167000E068012840F050813068216920F0F800CE
:1016800040EAC10030602078000713D4207840077A
:101690002AD4A569002D00F03A81B06800F00C0052
:1016A000082840F0A580012D40F00E81012002B0F5
:1016B000BDE8F0816069002800F082800020C4F25B
:1016C00047200121C0F8801EFFF7E2FD054600BF5C
:1016D000706F8007DAD4FFF7DBFD401B0228F7D9D3
:1016E000032002B0BDE8F081306C5FEAC0080AD484
:1016F00000200190306C40F080503064306C00F07D
:1017000080500190019847F20007C4F20007386842
:10171000C00547D4386840F480703860FFF7B8FDE2
:10172000054600BF3868C0053CD4FFF7B1FD401B3B
:101730000228F7D9032002B0BDE8F081B06800F0BC
:101740000C00082803D1706840023FF576AF61684D
:101750003068B1F5803F07D0B1F5A02F40F09A80F6
:1017600040F480203060306840F4803030609AE08F
:10177000E068002840F20000C4F247205CD001215C
:101780000160FFF785FD0546306880073FF574AFBF
:10179000FFF77EFD401B0228F6D9032002B0BDE80A
:1017A000F08100BFA168306F012905D0052955D10E
:1017B00040F004003067306F40F00100306756E0C1
:1017C0000020C4F247200021C0F8801EFFF760FD12
:1017D000054600BF706F80077FF558AFFFF758FDD3
:1017E000401B0228F6D9032002B0BDE8F08100BFFB
:1017F0000027C4F2472700203866FFF749FD022D75
:1018000005460DD13068800140F18A80FFF740FD28
:10181000401B02284FF00300F4D902B0BDE8F0816C
:101820003068800173D5FFF733FD401B02284FF06D
:101830000300F5D9F1E700BF00210160FFF728FDA3
:10184000054600BF306880077FF51DAFFFF720FD1C
:10185000401B02284FF00300F4D9DEE720F001001E
:101860003067306F002920F0040030677AD0FFF72E
:101870000FFD054641F28837306F800700F1848004
:10188000FFF706FD401BB842F6D9032002B0BDE8C1
:10189000F08100BF20F4803030603068002920F4EF
:1018A000802030607AD0FFF7F3FC05463068800373
:1018B0003FF5CAAEFFF7ECFC401B6428F6D90320C5
:1018C00002B0BDE8F08100BF7068E16900F48002F9
:1018D0008A4221D1216A00F03F028A421CD147F698
:1018E000C071626A0140B1EB821F15D1A16A4FF647
:1018F000FF73C903994300F44032A1F580318A4255
:101900000AD1E16A00F07060B0EB016F04D10020F1
:1019100002B0BDE8F08100BF012002B0BDE8F08157
:1019200004F11C052FCD084340EA8210D9034FF67D
:10193000FF729143A1F5803140EA05600843706071
:1019400001203866FFF7A4FC044600BF3068800120
:10195000DDD4FFF79DFC001B02284FF00300F5D9F2
:101960005BE700BFFFF794FC054641F2883700BFF4
:10197000306F800708D5FFF78BFC401BB8424FF053
:101980000300F5D949E700BFB8F1000F3FF581AE7C
:10199000306C20F0805030647BE600BFFFF778FCAD
:1019A000054600BF306880037FF54EAEFFF770FC40
:1019B000401B64284FF00300F4D92EE7411E00209D
:1019C000B0EB116F1CBF012070474EF21002CEF237
:1019D000000251604EF62351CEF20001F0230B704D
:1019E0000721906011607047704700007047000049
:1019F00090F83C20012A4FF0020254D010B580F834
:101A00003D200268D2F804E0D2F808C00C682EF03D
:101A10007003234341F2FF74C4F20004A2425360F6
:101A20000EDC40F2FF73C4F200039A4216DCB2F1FE
:101A3000804F2BD040F20043C4F2000324E000BFEB
:101A400040F2FF33C4F201039A4213DC41F6000373
:101A5000C4F200039A4219D0002313E040F60003B9
:101A6000C4F200039A4211D040F60043C4F20003CE
:101A70000AE000BF44F20003C4F201039A4205D019
:101A800040F20043C4F201039A4204D149682CF0A9
:101A90008003194391600121002280F83D1080F8F5
:101AA0003C20BDE81040104670470000002804BFED
:101AB0000120704710B5044690F83D0028B9002079
:101AC00084F83C00204600F01FF8022084F83D0016
:101AD0002068211D00F002FF012084F8460084F8F0
:101AE0003E0084F83F0084F8400084F8410084F808
:101AF000420084F8430084F8440084F8450084F8E8
:101B00003D00002010BD00000068B0F1804F18BFFC
:101B1000704780B582B00020019043F64000C4F2C7
:101B200002000168002241F001010160006800210B
:101B300000F00100019001981C20FFF743FC1C20DD
:101B400002B0BDE88040FFF72BBC000090F83D10CC
:101B500001291CBF01207047022180F83D10006858
:101B600041F2FF72C168C4F20002904241F00101EB
:101B7000C1600DDC40F2FF71C4F20001884215DC47
:101B8000B0F1804F2AD040F20041C4F2000123E0BE
:101B900040F2FF31C4F20101884213DC41F600013A
:101BA000C4F20001884219D0002113E040F6000180
:101BB000C4F20001884211D040F60041C4F2000195
:101BC0000AE000BF44F20001C4F20101884205D0DE
:101BD00040F20041C4F20101884206D1816801F05F
:101BE0000701062904BF00207047016841F0010188
:101BF000016000207047000090F83C20012A4FF05F
:101C000002026CD080B580F83D20D0F800C04FF6BD
:101C10007772DCF8083023EA0202CCF808200B685F
:101C20004F2B29DC1F2B45DD202B46D0302B44D0F9
:101C3000402B40F0AF80D1F804E0C968DCF82030D8
:101C4000DCF8202022F00102CCF82020DCF818205B
:101C500022F0F00242EA011123F00A0242EA0E02E7
:101C6000CCF81810CCF82020DCF8081041F047011F
:101C700021F0300128E000BF6F2B33DDB3F5005FAA
:101C800074D0B3F5805F21D0702B40F08380D1E910
:101C900001E3C968DCF8082043EA0E0322F47F421E
:101CA00043EA01211143CCF80810DCF8081041F098
:101CB000770109E00BB1102B6CD1DCF8081021F092
:101CC0007001194341F00701CCF8081000220121EE
:101CD00080F83D10002180F83C10BDE8804010469F
:101CE000704700BF502B21D0602B53D1D1F804E0B6
:101CF000C968DCF82030DCF8202022F01002CCF893
:101D00002020DCF8182022F4704242EA013123F04E
:101D1000A00242EA0E12CCF81810CCF82020DCF811
:101D2000081041F0670121F01001CDE7D1F804E07F
:101D3000C968DCF82030DCF8202022F00102CCF861
:101D40002020DCF8182022F0F00242EA011123F0F2
:101D50000A0242EA0E02CCF81810CCF82020DCF877
:101D6000081041F0570121F02001ADE7D1E901E36E
:101D7000C968DCF8082043EA0E0322F47F4243EAF4
:101D800001211143CCF80810DCF8081041F480411F
:101D90009AE700BF01229AE77047000070B5044639
:101DA0000068C5680669B10716D515F0020113D0A1
:101DB0006FF002010161012121778069800703D062
:101DC0002046FFF7E9FF05E0204600F08FF82046A7
:101DD00000F08EF800202077700719D515F0040068
:101DE00016D020686FF0040101610221217780691B
:101DF00010F4407F04D02046FFF7CEFF06E000BF7E
:101E0000204600F073F8204600F072F8002020779A
:101E1000300717D515F0080014D020686FF00801BE
:101E2000016104212177C069800703D02046FFF7B4
:101E3000B3FF05E0204600F059F8204600F058F8BE
:101E400000202077F00619D515F0100016D0206874
:101E50006FF01001016108212177C06910F4407F03
:101E600004D02046FFF798FF06E000BF204600F0B0
:101E70003DF8204600F03CF800202077F00718BF1E
:101E800015F0010002D1300609D412E020686FF08D
:101E900001010161204600F02DF8300609D515F04A
:101EA000800006D020686FF0800101612046FFF7B6
:101EB0009BFD700609D515F0400006D020686FF034
:101EC00040010161204600F045F8B00658BF70BDE2
:101ED00015F0200008D021686FF0200220460A612A
:101EE000BDE87040FFF782BD70BD00007047000084
:101EF0007047000080B582B00068B0F1804F01D01B
:101F000002B080BD01F0E6FF40F22010C2F20000F6
:101F1000416840F2DC520131914238BF0A460178F3
:101F20004378002918BF0022012B4260E8D1816864
:101F3000013164298160E3D34FF0080C00F10C03F8
:101F40000120022140F20972CDF800C0FEF724FB07
:101F500002B080BD70470000FEE7000080B540F28F
:101F6000C40046F20041C2F20000C4F2000140F891
:101F7000341F0C21002240F2001EC0E9011200F1C2
:101F80000C014FF420234FF4801CC0F2011E81E8A5
:101F90000C508283FEF744FE002808BF80BDBDE8D8
:101FA0008040FEF72DBB000070B586B0002543F6DB
:101FB00030000595CDE90355CDE901550095C4F2F2
:101FC00002000168002441F0800101600168C4F250
:101FD000020401F08001009100990095016800223F
:101FE00041F00101016001684FF4807601F00101C8
:101FF000009100990095016841F0020101600068BC
:102000004FF4807100F00200009000982046FFF726
:1020100039F90120CDE9020501A920460196049570
:10202000FFF760F806B070BD80B586B040F274204E
:102030000021C2F200004FF0804253234FF47A7C1B
:102040000591CDE90311CDE90011C0E90023C0E9F4
:10205000021C01618161FFF729FD002818BFFEF70E
:10206000CFFA4FF48050029040F27420C2F2000088
:1020700002A9FFF7C1FD002818BFFEF7C1FA40F220
:102080007420C2F200006946FFF7B2FC002818BFB6
:10209000FEF7B6FA06B080BDFEE70000FEE70000DE
:1020A00080B588B044F2C402C0F6000212688DF810
:1020B0000900079202AA032005927F228DF80A10D8
:1020C000ADF8180004A80DF107018DF8082001F003
:1020D00075FD08B080BD00007047000080B58EB06F
:1020E00001A9049140F20C61ADF80D1040F2080115
:1020F000C278C2F200010978772A18BF7622012936
:102100008DF80F2012D144F2C401C0F600014068DE
:10211000096800780D9108A90B917F218DF8201096
:102120008DF821008DF822103AE000BF0289416845
:10213000022A15D14878097800F07F02032A01D0DD
:10214000012A1DD140318DF804108DF805000221BF
:102150000006ADF814102BD403A80AA926E000BF8E
:1021600044F2C400C0F60000006809780D9008A889
:102170000B907F208DF820008DF8211013200DE0AA
:1021800044F2C400C0F6000000688DF821100D90E4
:1021900008A80B907F208DF8200012208DF82200D7
:1021A0000320ADF830000AA80DF11F0101F006FD73
:1021B0000EB080BD2DE9F04F91B000210991CDE91D
:1021C0000711CDE90511CDE90311CDE901118DF814
:1021D000031040F20C61ADF8191001A9C278079103
:1021E0004168772A18BF76228DF81B2011B1028929
:1021F000032A19D844F2C400C0F600000068109009
:102200000BA80E9043F27F10ADF82C0013208DF830
:102210002E000320ADF83C000DA80DF12B0101F0BC
:10222000CDFC11B0BDE8F08F4B7803F07F03012B9C
:102230001CD14B8840F202271BBA1B0CBB4249D071
:10224000B3F57F4F22D040F20327BB4262D1042A6C
:1022500058D140F22011C2F2000101220A7040F26E
:102260009001C2F2000100268E70BDE044F2C4006D
:10227000C0F600000068097810900BA80E907F202F
:102280008DF82C008DF82D101220C0E70D2A39D1C1
:10229000D1F8052040F2900413BAC2F20004A36101
:1022A000D1F809204CF20007C0F6000712BABB4271
:1022B000E2613FD1B2F5A82F3CD8054601200126A6
:1022C00000F07EFD01462846002940F08D80A67072
:1022D000002689E0082A15D140F210094968C2F2A7
:1022E0000009D9F8002009BA40F2900A8E1AC2F209
:1022F000000A18BF01269142CAF8201022D00126F8
:1023000072E000BF08781321FFF7CAFE11B0BDE8E4
:10231000F08F00BF44F2C400C0F6000000680978E6
:1023200010900BA80E907F208DF82C008DF82D10AA
:1023300031206CE708783121FFF7B2FE11B0BDE81B
:10234000F08F00BF0446012000F068FB6068A046E3
:10235000017842788378C07840318DF807000520F5
:102360008DF80410ADF8200006A80DF103018DF8DA
:1023700005208DF806308DF8086001F01FFCDAF8B2
:102380001C00800B14282DD84CF20004C0F6000469
:1023900000F0F6FCDAF81C104FF0FF30C9F800002E
:1023A00099B100274FF4A82B0DADE11911F80B10CE
:1023B00001228DF83410294600F084FCDAF81C1054
:1023C00001378F42C9F80000EFD3DAF820108142BC
:1023D00004D1022000F022FB04F5A824204601F0DD
:1023E000DBFD00E0002640464068017842788378B3
:1023F000C07840318DF8070005208DF80410ADF845
:10240000200006A80DF103018DF805208DF8063097
:102410008DF8086001F0D2FB11B0BDE8F08F00002C
:1024200070B58EB0018901AA0B2904924ED140F2F9
:102430009006C2F20006B2784068012A58D1B0F87E
:102440000120D0F8033032801ABAB260017AC37921
:10245000447A0904857A41EA036141EA04214B196F
:10246000D909F36001246D0618BF04EBD311316163
:102470004CF2000EC0F6000E90F800C0724547D135
:10248000002203EB0E01C0F60602914240D84078CC
:102490000CF140018DF8050080208DF80600032026
:1024A0008DF80410ADF81400022040F21001B07055
:1024B0000020C2F200014FF0FF32F0800A6070612C
:1024C00003A80AA901F07AFB0EB070BD44F2C40162
:1024D000C0F600014068096800780D9108A90B91C9
:1024E0007F218DF820108DF8210013201EE000BF01
:1024F00044F2C401C0F60001096800780D9108A9F2
:102500000B917F218DF820108DF8210024200DE003
:1025100044F2C400C0F6000000688DF821C00D90A0
:1025200008A80B907F208DF820001F208DF8220036
:102530000320ADF830000AA80DF11F0101F03EFBA9
:102540000EB070BD2DE9F047ADF5815D86B040F26B
:102550009009C2F20009824699F802000DF1060EB8
:102560000EF580580DF1040E0228DAF804000EF57D
:102570008051C8F80A101BD14178A9F8041069B33A
:10258000B9F8062001328A422CD1BAF80830A9F8ED
:102590000610032BA3F1020272D3D91E032902F005
:1025A000030C43D20023BCF1000F59D168E000BFF7
:1025B00044F2C401C0F60001096800780DF1080E6C
:1025C00004910EF581510DF5805E02917F218EF808
:1025D000290024208EF8281018E000BFB9F8062042
:1025E000FF2AD2D044F2C401C0F6000109680DF1FF
:1025F000080E007804910EF5815102917F210DF5AE
:10260000805E8EF828108EF8290073208EF82A003C
:102610000320ADF80C0001A80DF5815101F0CEFAB0
:102620000DF5815D06B0BDE8F08700BF22F0030123
:102630004E4201A9031F01316FF003059F794C1928
:10264000E770DF79043527711F7A67715F7A043389
:10265000A77177190437F1D12B1DBCF1000F0FD0F2
:102660000230C75C01A9BCF1010FCF5408D05F1C38
:10267000C65DBCF1020FCE5502D00233C05CC85417
:1026800040F21006C2F20006306801AD294600F0A3
:1026900019FB3060D9F80800D9F81410BAF80820EE
:1026A00000EBC110023A2946002300F051FE48B366
:1026B000DAF8040044F2C401C0F6000109680078A9
:1026C0000DF5805EC8F82E100DF581518EF82100B1
:1026D0007020C8F826107F218EF8220003208EF883
:1026E0002010AEF830000DF1080E0EF581500DF1FE
:1026F0001F0E0EF5805101F061FA0DF5815D06B0F7
:10270000BDE8F087D9F82400BAF808100DF5805E0E
:1027100008440238C9F82400DAF80400D9E90412A0
:102720000378407840338EF8043033688EF8050023
:1027300018BAC8F800000620AEF81400501C0DF1BD
:102740000C0EC9F81400022288420EF580500DF1DB
:10275000080E08BF032289F802200EF5815101F00E
:102760002DFA0DF5815D06B0BDE8F08710B58EB08D
:1027700001A90491018940F20C620129ADF80D20F4
:1027800018D140F29004C2F200044068A1780078A9
:10279000032921D140308DF804000120ADF8140048
:1027A00003A80AA901F00AFA0020A0706061E08085
:1027B0000EB010BD44F2C401C0F6000140680968C3
:1027C00000780D9108A90B917F218DF820108DF8CC
:1027D000210013200EE000BF44F2C401C0F6000146
:1027E00009688DF821000D9108A90B917F21242003
:1027F0008DF820108DF822000320ADF830000AA8D3
:102800000DF11F0101F0DAF90EB010BD70470000A4
:10281000FEF744BD70B592B006AC20463021FDF7FE
:10282000F6FD002543F640000595CDE90355CDE9B9
:1028300001550095C4F202000168022641F0805162
:102840000160006800F080500090009847F200009E
:102850000095C4F20000016841F480410160006805
:10286000A82100F4804000900098012006904FF4C9
:10287000803007904FF480000D9004200E9011904E
:1028800020460C96CDE90F16FEF7C2FE10B172B6C7
:10289000FEE700BF0F20CDE901064FF4A0500490E1
:1028A0004FF48050059001A805210395FEF7C6FD61
:1028B00010B172B6FEE700BF12B070BD4EF6885080
:1028C000CEF20000016841F4700101607047000021
:1028D00040F27420C2F20000FFF760BAB0B540F6D3
:1028E000FF3E0568C4F2000E40F2004C7045C4F291
:1028F000010C25DCB0F1804F2FD040F20043C4F230
:102900000003984229D040F60003C4F20003984225
:1029100023D041F6FF73C4F20003984228DC7045CF
:102920003ADCB0F1804F5BD040F20043C4F20003C8
:10293000984255D040F60003C4F200034EE000BFB9
:1029400040F60043C4F20003984206D0604504D02C
:102950000023C4F201039842DBD14B6825F07002DA
:1029600043EA020541F6FF73C4F200039842D6DD44
:1029700043F6FF73C4F2010398421FDC42F20003E6
:10298000C4F2000398422BD00023C4F20103984202
:1029900026D0604524D028E040F60043C4F200036E
:1029A00098421DD041F60003C4F20003984217D0AC
:1029B00041F60043C4F2000310E000BF44F20003FC
:1029C000C4F2010398420BD044F60003C4F20103A1
:1029D000984205D044F20043C4F20103984204D166
:1029E000CB6825F4407243EA02050A688C684B699B
:1029F000C46240F480648262644504BF0969016373
:102A0000026825F0800142F00402194302600122AD
:102A100042610160B0BD0000FEE7000070B582B009
:102A200043F6104648F20004C4F202060228C0F63B
:102A300000043FD0012840F08D8001208DF8060071
:102A400060788DF8070040F22310C4F2675046F812
:102A50000C0C48F6AB10CCF6EF5046F80C0CF320FB
:102A600046F8040C306820F440703060306840F460
:102A700000703060306820F078003060306840F0DE
:102A800012003060306840F480303060FEF700FCA7
:102A900056F8041CC90347D5054600BFFEF7F8FBEE
:102AA000401BB0F5FA6F46D856F8040CC003F5D4B5
:102AB0003AE000BF20788DF8060001208DF807006D
:102AC00040F22310C4F2675046F80C0C48F6AB10E5
:102AD000CCF6EF5046F80C0CF32046F8040C3068A6
:102AE00020F440703060306840F40070306030682E
:102AF00020F078003060306840F0120030603068BC
:102B000040F480303060FEF7C3FB56F8041CC90364
:102B10000AD50546FEF7BCFB401BB0F5FA6F0AD894
:102B200056F8040CC003F5D456F8040CC0071CBFBB
:102B3000012046F8040C30680DF1060120F07A00FF
:102B400030603068022240F00040306020460023B0
:102B500000F0FEFB02B070BD40F2B802C2F200020B
:102B6000135C002B04BF01207047B0B5135C02EB6F
:102B7000000C013B135440F234139CF8022000EB8C
:102B80008000C2F2000303EB401000EB0213D3E914
:102B900001454FEA021EDB68C1E9014550F80E000D
:102BA000CB600860501CC1B2092988BF00208CF896
:102BB00002000020B0BD000010B584B040F2B80E95
:102BC000C2F2000E1EF800C0BCF1090F24D81EF896
:102BD00000400EEB000C01340EF8004040F23414BB
:102BE00000EB8000C2F200049CF80AE004EB401005
:102BF0009CF80A4000EB0E1004F1010E5FFA8EF40F
:102C00000A2C8CF80AE024BF00248CF80A400160EA
:102C100003732BB914E000BF6846016003737BB1F6
:102C2000117801715178417191788171D178C171B8
:102C3000117901725179417291798172D179C172A0
:102C400004B010BD10B540F27804C2F20004207840
:102C500001281BD0A078012821D0E078012827D0B6
:102C60002079012805D10020207104F10800FFF728
:102C700069FC6079012818BF10BD002104F108002B
:102C80006171BDE81040FFF771BD00BF0021204613
:102C900000F8081BFFF722FAA0780128DDD10020F8
:102CA000A07004F10800FFF785FAE0780128D7D179
:102CB0000020E07004F10800FFF7B2FB2079012842
:102CC000D1D0D6E7002A08BF7047F0B502F0030C58
:102CD000940844F2CC024FF00003C0F600022AD060
:102CE000A3EB840E4C1C6FF0030300BFE518EE78D5
:102CF0002F794640F6B252F82660043386EA102057
:102D000087EA0006F6B252F826606F7986EA10204C
:102D100087EA0006F6B252F82660AD7986EA1020FE
:102D20004540EDB252F825500EEB0306043685EA15
:102D30001020DBD10433BCF1000F1DD0CF5CBCF1FF
:102D4000010F87EA0007FFB252F8277087EA1020C8
:102D500012D019444B78BCF1020F83EA0003DBB2B6
:102D600052F8233083EA102006D089784140C9B256
:102D700052F8211081EA1020BDE8F04070470000B1
:102D8000F0B581B0022000F01BF800244CF20007DF
:102D90004FF4A826C0F60604CFF6FA770DF1030526
:102DA000E05D29468DF8030020460122002300F053
:102DB000CFFA013E04F10104F2D101B0F0BD0000F0
:102DC0002DE9F04182B043F610460228C4F2020613
:102DD00000F03A81012840F03E8248F200040020D1
:102DE000C0F600048DF80600607848F6AB1840F293
:102DF0002317CCF6EF58C4F267578DF80700F3207D
:102E000046F80C7C46F80C8C46F8040C306820F42C
:102E100040703060306840F400703060306820F0FE
:102E200078003060306840F012003060306840F464
:102E300080303060FEF72CFA56F8041CC9030BD51D
:102E4000054600BFFEF724FA401BB0F5FA6F0AD81A
:102E500056F8040CC003F5D456F8040CC0071CBF88
:102E6000012046F8040C30680DF1060120F07A00CC
:102E700030603068022240F000403060204600237D
:102E800000F066FAF32046F80C7C46F80C8C46F805
:102E9000040C306820F440703060306840F40070FA
:102EA0003060306820F078003060306840F01A0000
:102EB0003060306840F480303060FEF7E9F956F851
:102EC000041CC9030AD50446FEF7E2F9001BB0F55D
:102ED000FA6F0AD856F8040CC003F5D456F8040C5F
:102EE000C0071CBF012046F8040C306820F07A00AF
:102EF0003060306840F000403060F32046F80C7CD1
:102F000046F80C8C46F8040C306820F440703060B1
:102F1000306840F400703060306820F07800306035
:102F2000306840F022003060306840F4803030601B
:102F3000FEF7AEF956F8041CC9030BD5044600BFD2
:102F4000FEF7A6F9001BB0F5FA6F0AD856F8040C84
:102F5000C003F5D456F8040CC0071CBF012046F886
:102F6000040C306820F07A003060306840F0004097
:102F70003060F32046F80C7C46F80C8C46F8040CC4
:102F8000306820F440703060306840F40070306089
:102F9000306820F078003060306840F02A003060FF
:102FA000306840F480303060FEF772F956F8041C47
:102FB000C9030BD5044600BFFEF76AF9001BB0F544
:102FC000FA6F0AD856F8040CC003F5D456F8040C6E
:102FD000C0071CBF012046F8040C306820F07A00BE
:102FE0003060306840F000403060F32046F80C7CE0
:102FF00046F80C8C46F8040C306820F440703060C1
:10300000306840F400703060306820F07800306044
:10301000306840F032003060306840F4803030601A
:10302000FEF736F956F8041CC90340F10581044641
:10303000FEF72EF9001BB0F5FA6F00F2048156F886
:10304000040CC003F4D4F7E048F20004C0F6000416
:10305000207848F6AB1840F223178DF806000020C0
:10306000CCF6EF58C4F267578DF80700F32046F806
:103070000C7C46F80C8C46F8040C306820F4407048
:103080003060306840F400703060306820F07800C4
:103090003060306840F012003060306840F48030BA
:1030A0003060FEF7F5F856F8041CC9030AD505464A
:1030B000FEF7EEF8401BB0F5FA6F0AD856F8040C8C
:1030C000C003F5D456F8040CC0071CBF012046F815
:1030D000040C30680DF1060120F07A003060306891
:1030E000022240F0004030602046002300F030F91A
:1030F000F32046F80C7C46F80C8C46F8040C30683B
:1031000020F440703060306840F400703060306807
:1031100020F078003060306840F03A00306030686D
:1031200040F480303060FEF7B3F856F8041CC90351
:103130000AD50446FEF7ACF8001BB0F5FA6F0AD8C2
:1031400056F8040CC003F5D456F8040CC0071CBF95
:10315000012046F8040C306820F07A0030603068B6
:1031600040F000403060F32046F80C7C46F80C8CB0
:1031700046F8040C306820F440703060306840F449
:1031800000703060306820F078003060306840F0C7
:1031900042003060306840F480303060FEF778F8EC
:1031A00056F8041CC9030BD5044600BFFEF770F89F
:1031B000001BB0F5FA6F0AD856F8040CC003F5D41A
:1031C00056F8040CC0071CBF012046F8040C3068F8
:1031D00020F07A003060306840F000403060F3202A
:1031E00046F80C7C46F80C8C46F8040C306820F449
:1031F00040703060306840F400703060306820F01B
:1032000078003060306840F04A003060306840F448
:1032100080303060FEF73CF856F8041CC9030BD52B
:10322000044600BFFEF734F8001BB0F5FA6F0AD869
:1032300056F8040CC003F5D456F8040CC0071CBFA4
:10324000012046F8040C306820F07A0030603068C5
:1032500040F000403060002002B0BDE8F081000086
:10326000B0B543F6104540F22311C4F20205C4F292
:10327000675145F80C1C48F6AB11CCF6EF5145F8F8
:103280000C1C4FF6FF7120EA0101B1F1006F4FF005
:10329000F30145F8041C05D1182101EAD0200230C1
:1032A00020E000BF40F60101B1EB104F02D1222017
:1032B00018E000BF0021CFF2FE714218B2F5202FB6
:1032C00004D2382000EA92302A300BE00022C0F607
:1032D000010201F10061014002F530225A209142C1
:1032E00008BF5220296821F440712960296841F4FF
:1032F00000712960296821F0780129602968084354
:103300002860286840F480302860FDF7C1FF55F838
:10331000041CC9030AD50446FDF7BAFF001BB0F52B
:10332000FA6F0AD855F8040CC003F5D455F8040C0C
:10333000C0071CBF012045F8040C286820F07A0063
:103340002860286840F0004100202960B0BD0000DE
:103350002DE9F04791460D46074600F0030620F0A0
:10336000030813B14046FFF77BFF43F6104440F2D9
:103370002310C4F20204C4F2675044F80C0C48F65F
:10338000AB10CCF6EF5044F80C0CF320002E44F8B0
:10339000040C18BFB9F1000F00F093802878216861
:1033A00021F44071216021682160216841F0010110
:1033B00021603870FDF76CFF54F8041CC9030AD56E
:1033C000074600BFFDF764FFC01B0A280AD854F85F
:1033D000040CC003F6D454F8040CC0071CBF012031
:1033E00044F8040C2068691C20F001002060701C67
:1033F0008207A9F1010218BF002A5FD0097822686C
:1034000022F44072226022682260226842F00102A7
:10341000226000F80810FDF73BFF54F8041CC903B4
:1034200009D50746FDF734FFC01B0A280AD854F80F
:10343000040CC003F6D454F8040CC0071CBF0120D0
:1034400044F8040C2068A91C20F001002060B01C86
:103450008207A9F1020218BF002A2FD0097822683A
:1034600022F44072226022682260226842F0010247
:10347000226000F80810FDF70BFF54F8041CC90384
:1034800009D50746FDF704FFC01B0A280AD854F8DF
:10349000040CC003F6D454F8040CC0071CBF012070
:1034A00044F8040C2068E91C20F001002060F01CA6
:1034B0008207A9F1030218BF002A3BD10D469146AD
:1034C0000646B9F1040F64D34FF0010A12E000BFC1
:1034D00054F8040CC00718BF44F804AC2068A9F1E4
:1034E000040920F001000435B9F1030F06F10406C8
:1034F00020604ED92868216821F44071216021683C
:1035000041F400712160216841F00101216046F819
:103510000800FDF7BDFE54F8041CC903D8D50746C2
:10352000FDF7B6FEC01B0A28D8D854F8040CC00317
:10353000F6D4CDE70978226822F44072226022682E
:103540002260226842F00102226000F80810FDF7B4
:103550009FFE54F8041CC90309D50746FDF798FEE1
:10356000C01B0A280AD854F8040CC003F6D454F837
:10357000040CC0071CBF012044F8040C206804356B
:1035800020F0010020600436A9F10409B9F1040F0C
:103590009AD2B9F1000F31D04FF0010A10E000BF0C
:1035A00054F8040CC00718BF44F804AC2068013577
:1035B00020F00100B9F1010906F1010620601DD0DB
:1035C0002878216821F440712160216821602168F8
:1035D00041F00101216006F80800FDF759FE54F89A
:1035E000041CC903DCD50746FDF752FEC01B0A28A0
:1035F000DCD854F8040CC003F6D4D1E7206840F0BE
:10360000004100202160BDE8F087000040F2BC20AE
:10361000C2F200000021017540F6D420C2F2000081
:103620000176C1617047000070B586B040F2BC24DD
:10363000C2F200042179027891420BD1617942787B
:10364000914207D1E179C278914203D100212175DD
:1036500004E000BF217D09B106B070BD4268117859
:10366000537801F00F0143EA01210829F4D30389BB
:103670000232023B00264260038126708368C4E95F
:103680000223C26803682261A18102896360002A63
:1036900004F11802A26032D0002100BF4368CAB210
:1036A000A5689A5C6B1CA3602A7041F00102038933
:1036B000D2B2934222D94368A5689A5C6B1CA3607E
:1036C0002A7041F002020389D2B2934216D94368AC
:1036D000A5689A5C6B1CA3602A7041F00302038901
:1036E000D2B293420AD94368A5689A5C6B1CA36066
:1036F0002A7004310289CBB29A42CFD8A18944F210
:10370000B800C0F600000088B1F5006FE0824FF00D
:1037100006004FF0300188BF072088BF32218DF8A6
:10372000001044F2B00120756846C0F60001039015
:1037300044F2AC000978C0F6000000788DF8021061
:1037400040F21401C2F200018DF801000320097853
:10375000ADF8100020798DF80810E1888DF8090087
:1037600002A8ADF80A1000F095F944F2B200C0F6D4
:1037700000000088217DE082062908BF0526267505
:1037800006B070BD70B584B00368017B40F2DF7491
:10379000021DA3424FF000040192ADF808108DF80D
:1037A000024007D177238DF80330F1238DF80030E4
:1037B00011E000BF44F2C004C0F600042468A34234
:1037C00009D176248DF80340F1248DF8004021338F
:1037D00001248DF801301278D3B20022102B38BFAB
:1037E00001222243D2070BD03F2B09D81A09DFE868
:1037F00002F00351091B00BF002B18BF99424FD89C
:1038000004B070BD40F2BC24C2F20004227D052A3F
:10381000F6D12278013253401B0722704AD0002093
:10382000207504B070BD00BF40F6D422C2F2000281
:10383000167E042EE4D10329E2D303F00F010129FF
:1038400052D000295FD103211176417990F9060009
:103850006FF0F00353FA80F3092B4FF07F0338BF6A
:103860000123002858BFC3B244F2AE00C0F60000E6
:1038700000781170517044F2B401B3FBF0F0C0F65F
:10388000000109885080908000201184D07104B01C
:1038900070BD00BF6846FFF7C7FE04B070BD00BF33
:1038A000053001906846ADF8083000F023FB04B005
:1038B00070BD00BFB4F80CC0A26804EB0C039B1AE7
:1038C000A1F1010E03F118011FFA8EF389B299429A
:1038D00038BF0B46D9B2002961D0042903F0030C8C
:1038E0001ED200213EE000BF0420107644F2B60054
:1038F000C0F600000088D1791084481CC1B20529A7
:10390000D071FFF47DAF00201076D06902210170E4
:1039100040F6F860C2F20000D06104B070BD00BF94
:10392000021FACEB010E6FF0030300BFA168557AD4
:103930004E1CA6600D70A168957A4E1CA6600D7095
:10394000A168D57A4E1CA6600D70A168157B4E1C2F
:103950000433A6600D700EEB0301043102F1040282
:10396000E4D1191DBCF1000F16D00530A268435CEC
:10397000561CBCF1010FA66013700DD00844A1685D
:1039800042784B1CBCF1020FA3600A7004D0A168FE
:1039900080784A1CA2600870B4F80CC0A26804EBDE
:1039A0000C00801A1830000408D044F2B200C0F6AF
:1039B00000000088E08204B070BD00BF04F1180070
:1039C000A060201D00F096FA0020207504B070BDA4
:1039D00010B58AB069460020FFF7BEF848B96C46BA
:1039E0002046FFF7CFFE00202146FFF7B5F800285C
:1039F000F6D040F2BC24C2F20004207D00F0FE00AC
:103A000006283DD1A0890621B0F5006F88BF0721A7
:103A10004FF0300088BF3220217504A9079144F28D
:103A2000B001C0F600018DF8100044F2AC00097836
:103A3000C0F6000000788DF8121040F21401C2F2B6
:103A400000018DF8110003200978ADF820002079DD
:103A50008DF81810E1888DF8190006A8ADF81A1035
:103A600000F018F844F2B200C0F600000088217D92
:103A70000022E082062908BF0522227501E000BF6E
:103A8000E08A002807BF002020750138E0820AB0D4
:103A900010BD000080B586B044F2C401C0F600013C
:103AA000B0F808C00A6802ABBCF1000F03F10403D0
:103AB000029235D04168BCF1010F09788DF80C10E5
:103AC00035D04168BCF1020F49788DF80D1035D919
:103AD0004168BCF1030F89788DF80E1035D041682C
:103AE000BCF1040FC9788DF80F1035D94168BCF1CD
:103AF000050F09798DF8101035D04168BCF1060F1B
:103B000049798DF8111035D94168BCF1070F8979D1
:103B10008DF812104ED144F2AD00C0F6000030E036
:103B200044F2AD00C0F6000000788DF80C0044F2BD
:103B3000AD00C0F6000000788DF80D0044F2AD0035
:103B4000C0F6000000788DF80E0044F2AD00C0F61B
:103B5000000000788DF80F0044F2AD00C0F60000C0
:103B600000788DF8100044F2AD00C0F60000007837
:103B70008DF8110044F2AD00C0F6000001788DF818
:103B80001210007844F2C8018DF8130044F2BC0012
:103B9000C0F60000C0F60001007809684FF0080C7C
:103BA0008DF814C0CDF800C0FCF7F6FC002006B07C
:103BB00080BD00BF40680730E3E7000070B586B005
:103BC00040F6F866C2F20006002918BF0E4640F221
:103BD0001401C2F2000102890978072A017031D864
:103BE00090E82A00C468002A8DE82A0003948DF822
:103BF000102000F09D804068D1B201320378022A83
:103C00008DF811301BD04378032A8DF8123016D06E
:103C10008378042A8DF8133011D0C378052A8DF8E3
:103C200014300CD00379062A8DF8153007D043796B
:103C3000072A8DF816301CBF80798DF81700481CB4
:103C400077E000BF0221B2F5806F31706DD840F689
:103C5000D425C2F20005297E002966D14FF0010C5F
:103C600086F800C002892AB3002200BF4368511CB5
:103C70009C5CAB1883F822400489A1421AD24168A7
:103C8000941C1144497883F8231001898C4211D285
:103C90004168D41C1144897883F8241001898C422E
:103CA00008D241681144C978043283F8251001898B
:103CB0008A42DBD390E80E00C06805F1080E8EE85A
:103CC0000E006861CDE9023004A80190288A05F150
:103CD000220200911021EA6044F2BA0241EA102166
:103CE0008DF81100D5F82200C0F6000212888DF878
:103CF0001010E98CCDF812000820ADF808006846D5
:103D000085F818C085F806C0EE612A84ADF8161053
:103D1000FFF7C0FE44F2B601C0F600010420098896
:103D2000287605F128002984E86006B070BD00BF40
:103D3000012004A9ADF8080068460191FFF7AAFE2A
:103D40000020307006B070BDB0B586B040F6D42407
:103D5000C2F20004207E03283AD0012840F0B1804E
:103D6000A068D4E90412009004A8CDE902120190E1
:103D7000208A102141EA10218DF81100E08CD4F83E
:103D80002230ADF816000820ADF8080068468DF81E
:103D90001010CDF81230FFF77DFE44F2B600C0F6E9
:103DA000000004210088217604F128012084E160CC
:103DB000002840F08A8000202076E069022101700E
:103DC00040F6F860C2F20000E06106B0B0BD00BF8E
:103DD000D4E90401A268CDE90201A08804A90092F7
:103DE000019118B10138A0806BE000BF6088A17913
:103DF000A080481CE568A071022060F31F11208A92
:103E00008DF81010611B0844223080B2072828BFAB
:103E10000720002800F1010033D0294611F8012BBA
:103E200002288DF811202BD0697803288DF8121004
:103E300002D1A91C24E000BFA97804288DF8131032
:103E400002D1E91C1CE000BFE97805288DF81410A8
:103E500002D1291D14E000BF297906288DF815101C
:103E600002D1691D0CE000BF697907288DF8161092
:103E700002D1A91D04E000BFAA79E91D8DF8172021
:103E80000D46C0B2ADF808006846FFF703FE44F2E5
:103E9000B400C0F6000000882A1B218A223A208440
:103EA000607892B29142A0F10100E560607008D1A3
:103EB000E0690021017040F6F860C2F20000E061A4
:103EC0002176208C00283FF476AF0138208406B09C
:103ED000B0BD000080B5FFF77BFDBDE88040FFF777
:103EE00033BF000040F20800C2F20000022101705E
:103EF0007047000070B50446028940F27806C06839
:103F000040F6FC65C2F200066168C2F2000570610D
:103F100028463282FCF736FAF56060680078A0F136
:103F20001101262922D8DFE801F0152121212121C4
:103F30002121212121212121212121212121212171
:103F4000212121212121212B21211921212F21333F
:103F50001D0000BF0120307070BD00BF0120B07097
:103F600070BD00BF0120707170BD00BFE17876297F
:103F700018BF70BD1121BDE87040FEF791B800BFB9
:103F80000120707070BD00BF0120F07070BD00BFD7
:103F90000120307170BD000010B504464EF21000D3
:103FA000CEF200000021016040F2F800C2F20000F1
:103FB000FCF730FCFCF78AFF206880F308884EF697
:103FC0000850CEF2000004606068BDE81040004771
:103FD00082B048F20006C0F60006FDF76DF9FEF764
:103FE00019FCFDF7E1FFFDF7B9FFFEF71DF840F200
:103FF0007420C2F20000FDF7A9FDFCF7A7FAFFF755
:1040000005FBFFF76FFF40F22C1342F20120C2F2D2
:104010000003C4F23340186046F25560C8F67700DA
:104020005860082000900120022140F209724FF0F0
:104030000108FCF7B1FA40F2241740F2211AC2F24B
:10404000000740F2DC5506F5804406F5B029C2F2BF
:10405000000A03E020463D60FFF79EFFFEF7F2FDF9
:104060003868A842FAD130780128F3D07078012856
:1040700004D148463D60FFF78FFFEFE78AF80080E4
:10408000ECE7F1EE100A4FF6FF71C0F2C03120EA02
:10409000010040F04070E1EE100A7047000000009F
:1040A0000000000001020304060708090055010092
:1040B0000100960046009600460046000000000001
:1040C00001070000090700000000000000000000D8
:1040D000963007772C610EEEBA51099919C46D0715
:1040E0008FF46A7035A563E9A395649E3288DB0E70
:1040F000A4B8DC791EE9D5E088D9D2972B4CB60953
:10410000BD7CB17E072DB8E7911DBF906410B71D2F
:10411000F220B06A4871B9F3DE41BE847DD4DA1A68
:10412000EBE4DD6D51B5D4F4C785D38356986C1399
:10413000C0A86B647AF962FDECC9658A4F5C011412
:10414000D96C0663633D0FFAF50D088DC8206E3BF0
:104150005E10694CE44160D5727167A2D1E4033C02
:1041600047D4044BFD850DD26BB50AA5FAA8B53529
:104170006C98B242D6C9BBDB40F9BCACE36CD83218
:10418000755CDF45CF0DD6DC593DD1ABAC30D926BF
:104190003A00DE518051D7C81661D0BFB5F4B421C2
:1041A00023C4B3569995BACF0FA5BDB89EB80228BF
:1041B0000888055FB2D90CC624E90BB1877C6F2F44
:1041C000114C6858AB1D61C13D2D66B69041DC763F
:1041D0000671DB01BC20D2982A10D5EF8985B17118
:1041E0001FB5B606A5E4BF9F33D4B8E8A2C90778C7
:1041F00034F9000F8EA8099618980EE1BB0D6A7F5E
:104200002D3D6D08976C6491015C63E6F4516B6B16
:1042100062616C1CD83065854E0062F2ED95066CCB
:104220007BA5011BC1F4088257C40FF5C6D9B06540
:1042300050E9B712EAB8BE8B7C88B9FCDF1DDD629D
:10424000492DDA15F37CD38C654CD4FB5861B24D03
:10425000CE51B53A7400BCA3E230BBD441A5DF4ACD
:10426000D795D83D6DC4D1A4FBF4D6D36AE9694390
:10427000FCD96E34468867ADD0B860DA732D04443B
:10428000E51D03335F4C0AAAC97C0DDD3C71055066
:10429000AA41022710100BBE86200CC925B568570D
:1042A000B3856F2009D466B99FE461CE0EF9DE5E56
:1042B00098C9D9292298D0B0B4A8D7C7173DB35907
:1042C000810DB42E3B5CBDB7AD6CBAC02083B8ED98
:1042D000B6B3BF9A0CE2B6039AD2B1743947D5EAA5
:1042E000AF77D29D1526DB048316DC73120B63E3D4
:1042F000843B64943E6A6D0DA85A6A7A0BCF0EE433
:104300009DFF099327AE000AB19E077D44930FF0ED
:10431000D2A3088768F2011EFEC206695D5762F7E4
:10432000CB67658071366C19E7066B6E761BD4FE21
:10433000E02BD3895A7ADA10CC4ADD676FDFB9F9FE
:10434000F9EFBE8E43BEB717D58EB060E8A3D6D6C0
:104350007E93D1A1C4C2D83852F2DF4FF167BBD1EE
:104360006757BCA6DD06B53F4B36B248DA2B0DD8F1
:104370004C1B0AAFF64A0336607A0441C3EF60DF94
:1043800055DF67A8EF8E6E3179BE69468CB361CB7D
:104390001A8366BCA0D26F2536E2685295770CCCA2
:1043A00003470BBBB91602222F260555BE3BBAC5E3
:1043B000280BBDB2925AB42B046AB35CA7FFD7C2D4
:1043C00031CFD0B58B9ED92C1DAEDE5BB0C2649BC5
:1043D00026F263EC9CA36A750A936D02A906099CF8
:1043E0003F360EEB8567077213570005824ABF956B
:1043F000147AB8E2AE2BB17B381BB60C9B8ED292EE
:104400000DBED5E5B7EFDC7C21DFDB0BD4D2D38644
:1044100042E2D4F1F8B3DD686E83DA1FCD16BE81B7
:104420005B26B9F6E177B06F7747B718E65A088888
:10443000706A0FFFCA3B06665C0B0111FF9E658F19
:1044400069AE62F8D3FF6B6145CF6C1678E20AA0C3
:10445000EED20DD75483044EC2B30339612667A749
:10446000F71660D04D476949DB776E3E4A6AD1AE98
:10447000DC5AD6D9660BDF40F03BD83753AEBCA927
:10448000C59EBBDE7FCFB247E9FFB5301CF2BDBD94
:104490008AC2BACA3093B353A6A3B4240536D0BA9D
:1044A0009306D7CD2957DE54BF67D9232E7A66B33A
:1044B000B84A61C4021B685D942B6F2A37BE0BB4E7
:1044C000A18E0CC31BDF055A8DEF022D00010403E2
:1044D000F04400080000002018000000EC01000873
:1044E0000845000818000020E82400000C0200081D
:1044F0000100000010000000020000000024F40091
:08450000FFFFFFFFF1000000C6
:040000050800018965
:00000001FF
